:0800000000308B000D108D1083
:08000800850186018316073013
:0800100081001F3085000F3054
:0800180086000230880083120B
:08002000C13088007F308E0022
:080028008F008E2820308C00AF
:080030008C0B18280800A63013
:080038008C008C0B1D28080050
:0800400016200815162008190E
:080048002328090892000800BA
:0800500006080F390319013005
:0800580090000800100891005F
:080060000D08013A8D000D1C92
:0800680039280608203A860041
:080070003D28861E0612861AC7
:0800780006161B20910B302835
:080080008E0312080E06031D99
:080088002E2808001008910069
:080090000D08013A8D000D1C62
:0800980051280608203A8600F9
:0800A0005528861E0616861A7B
:0800A80006121B20910B4828F1
:0800B0008E0A12080E06031D62
:0800B800462808001008910021
:0800C0000D08023A8D008D1CB1
:0800C80069280608803A860051
:0800D0006D28861F0613861B34
:0800D80006171B20910B6028A4
:0800E0008F0A12080F06031D30
:0800E8005E28080010089100D9
:0800F0000D08023A8D008D1C81
:0800F80081280608803A860009
:080100008528861F0617861BE7
:0801080006131B20910B78285F
:080110008F0312080F06031D06
:08011800762808000D152820CF
:0801200088112020051D9F2815
:0801280012080E020319A028C1
:08013000031C0D110D1D4620FA
:080138000D192E20A0288E00F5
:080140000D1528208815202070
:08014800051DB12812080F0289
:0801500003198E28031C0D1198
:080158000D1D5E200D1976203B
:060160008E288F008E289E
:00000001FF
